:080000000C946D010C94580BE7
:100008000C9400000C9400000C9400000C94000068
:100018000C9400000C9400000C9400000C94000058
:100028000C9400020C9400000C9400000C94000046
:100038000C9400000C9400000C94A3010C94000094
:100048000C94B5080C9400000C9401090C94000061
:100058000C9400000C9400000C9400000C94000018
:100068000C9400000C9400000C9400000C94000008
:100078000C942B0A0C9400000C940F0B0C940000A9
:100088000C94000000010204081020408000680160
:100098000000801002006C011500011000007A01B8
:1000A80013000101000082010100010200008C011F
:1000B8000200010200009601030001020000A001F5
:1000C800040001020000AA01050001020000B401B9
:1000D800060001020000BE01070001020000C8017D
:1000E800080001020000D201090001020000DC0141
:1000F8000A0001020000E6010B0001020000F00105
:100108000C0001020000FA010D00010200000402C7
:100118000E00010200000E020F000102000018028A
:1001280010000102000022021100010200002C024E
:1001380012000102000000000000FF0000000000A3
:1001480001000200040008001000200040008000A8
:100158000001000200040008001000200040008098
:100168005F4944005F53656E64496E707574546FDF
:1001780000005F52656C616973005F496E70757449
:100188005F3100005F496E7075745F3200005F492F
:100198006E7075745F3300005F496E7075745F34FC
:1001A80000005F496E7075745F3500005F496E70BE
:1001B80075745F3600005F496E7075745F370000B4
:1001C8005F496E7075745F3800005F496E707574B2
:1001D8005F3900005F496E7075745F3130005F49A8
:1001E8006E7075745F3131005F496E7075745F3180
:1001F80032005F496E7075745F3133005F496E700D
:1002080075745F3134005F496E7075745F31350005
:100218005F496E7075745F3136005F496E70757432
:100228005F3137005F496E7075745F313800102791
:10023800E80364000A00010000100001100001003A
:1002480049530049430025642E2532640044530075
:10025800564300494C0023502241534349492D49F4
:100268002F4F222C22312E3030222C323030382D94
:1002780030312D30313B0023482245636F222C2238
:10028800312E3030222C323030382D30312D303173
:100298003B0023532245636F222C22312E3030221B
:1002A8002C323030382D30312D30313B0000256470
:1002B800002530325800253130640000564300498B
:1002C800500001002D4E414E00000100E00FCA020F
:1002D8000000F894EE27ECBBF1E0F5BFE5BFE09332
:1002E8006C00F8E1F1BDE1BD8DE0A2E0BB27ED9324
:1002F8008A95E9F780E090E1A0E0B1E0ED930197FD
:10030800E9F7E2EDF2E085919591009761F0A5910A
:10031800B59105901590BF01F00105900D920197D8
:10032800E1F7FB01F0CFEFEFEDBFE0E1EEBFC0E09A
:10033800D5E00C944C03E0916300E07108950E94AD
:10034800D712E4E6E2BF0E94FD034394E2E3E4151A
:1003580019F4E1E0E71509F002C077244424E2E348
:10036800E41519F4E0E0E71509F003C0E1E07E2E9A
:100378004424A0910105A13028F0E0910105E15045
:10038800E0930105E6B3E093920BA3E9BBE0E0B18B
:10039800EC93E0B3E073E295EF70E093940B0E9466
:1003A8006D0EA091DF0CB091E00CEFEFF0E0EA27C2
:1003B800FB27EBBBE091DF0CF091E00C0E943115BC
:1003C800AFEFB0E0EA27FB27E5BBA3E1B0E00E946E
:1003D800A515E13031F4E091DF0CF091E00CE1700B
:1003E80009F404C0E0916500E26003C0E091650093
:1003F800ED7FE093650017C00E94D7121A930A9305
:10040800E6E0E4BDE6B3F0E0DF01E0B1FE2FE0E0B6
:10041800EA0FFB1F8F011A930A930E94E00D0E94B6
:10042800930D09911991E991EFBFF991E991B9916A
:10043800A9919991899179916991F9901990099067
:1004480018951A93A0915808A13051F4DA92CA92DB
:10045800E4E6F0E0FA93EA930E943004E03009F40D
:1004680009C0E0E0E0935808E3E0E91518F40E94B9
:10047800E5129924A0915808A23041F4DA92CA9260
:100488000E94ED120E943004E03009F403C0E0E05D
:10049800E0935808A0915808A03059F4E09151060B
:1004A800A0915206EA1729F0A0E020FCA1E0A030B4
:1004B80009F027C00E94F212EE5FFA4FE081E130A6
:1004C80039F40E94F2120E94F8120E94FF1219C019
:1004D800E23011F0E330A9F40E94F212EE5FFA4F15
:1004E800E081E23009F499240E94F2120E94F81285
:1004F800EE5FFA4FA3E0A083A3D16F01E1E0E093A0
:1005080058080C94FC041A93A0915506A43011F4D1
:1005180010918A07A0915506A53011F41091F107A2
:10052800143049F4E981E03011F4E0E001C0EFE073
:10053800EA930E947C04153049F4E981E03011F413
:10054800E5E101C0E6E0EA930E947C0462C01A93E8
:10055800E3E0EA930E947C0410915406E12FE295AF
:10056800EF700E940413E12FEF700E940413E7E17B
:10057800EA930E947C040C94FC04E2E0EA930E9453
:100588007C04E0E0E0935406E9E4EA930E947C04EA
:10059800E881E05DEA930E947C04D9DFA0915506CA
:1005A800A43011F40E940A130E9411131696E1E078
:1005B800EC93E8810E9416130C94D3041A93A0912B
:1005C8005506A43011F40E940A1310E0173060F4A5
:1005D8000E9411131A96EE27A10FBE1FEC91EA9301
:1005E8000E947C041F5FF2CFE981E03011F4E0E360
:1005F80005C0E091060DF091070DE189EA930E948C
:100608007C040E9411131696E1E0EC93E9810E94A4
:100618001613188122960895E0915906A09158065C
:10062800EA1759F0A0915706A13039F40E94F00852
:10063800EB3018F080DEE03009F40FC0E091590685
:10064800F0E0E65AF94FE081EA930E943109A0915F
:1006580059060E941D13E093590608951A93A89508
:100668000E940D0D0E94D70CECDED6DFE0E0E71506
:1006780021F4A0910105A03021F0E0916500EE7F02
:1006880003C0E0916500E160E09365000C94FC0410
:10069800E0E0E5BFE0936D00E0936C00EFEFEBBBAB
:1006A800EABBE0E0E8BBE7BBEFEFE5BBE4BBE0E0BB
:1006B800E2BBE1BBE3B9E2B9E0936200E093610019
:1006C800E0936500E3E0E0936400E0E0E0BFE7E08A
:1006D800E3BFE4E6E2BFE0E0E1BFEFBDEEBDEDBDA4
:1006E800ECBDE7BDE6BDEBBDEABDE9BDE8BDE09305
:1006F8007900E0937800E3E0E5BDE6E0E4BDE0E002
:10070800E3BDE0938B00EAE0E0938A00E0E0E09349
:100718008900E0938800E0938100E0938000E2E1A3
:10072800E0938700E4E3E0938600E0E0E09385004F
:10073800E0938400E0938300E0938200E0936A00F2
:10074800EABFE9BFE1E4E7BFE0E0E0937D00EBB991
:10075800E8EDEAB9E6E0E0939500E0E0E093900088
:10076800E6E6E9B9E0E0E0939B00E8EDE0939A0063
:10077800E6E0E0939D00E0E0E0939800E3E3E09397
:100788009900E0E8E8B9E0E0E0BDEEE1E1BDEEE0C7
:10079800E1BD0E9490080E94C0100E942213E5311A
:1007A80028F0A0E0B0E0E0E00E94B91588240E949B
:1007B80022138E1668F4A895E0916500EE7F0E94DA
:1007C8002713E0916500E1600E9427138394EFCF1F
:1007D800E8ECF0E0FA93EA930E9416157894EFEFAC
:1007E8006E2E3CDF0E948410E1E0E0935706F9CFBB
:1007F800FFCFA8E0BDE00E942F130895A881A03381
:1008080010F0AA3308F003C0E881E053C8C0A881FB
:10081800A13410F0A73408F003C0E881E753BFC043
:10082800EFEFBDC0A881AA3018F4E881E05DB7C039
:10083800A881AA3018F0E881E95CB1C0E8E5AFC04A
:100848001A930A93F8940091080D1091090D789461
:10085800F8010991199108951A930A93F1DF8F010C
:10086800EA81FB81AC81BD81EA0FFB1FE01BF10B24
:10087800DF010E94CA1524F4E0E019810881BFC293
:10088800E1E019810881BBC2E881EF5FE883A881B4
:10089800A53010F0E0E0E883E88181C0A09152061D
:1008A800BB27E0915106F0E031960E94351335964A
:1008B800DF01E5E0F0E00C94FE08A0915906BB27A3
:1008C800E09158060C94F508A0915306A13059F40C
:1008D800A0915706A13039F4F0DFE93220F00E94E8
:1008E8009F01E03009F402C0E1E00895E0E00895D6
:1008F800E881A0915406EA27E0935406E091550652
:10090800E13071F4E0915806F0E0E65AF94FA88119
:10091800A083A09158060E941D13E09358063FC07B
:10092800E23071F4E091BE06F0E0E054F94FA8819E
:10093800A083A091BE060E941D13E093BE062FC09F
:10094800E33071F4E0912407F0E0EA5DF84FA88104
:10095800A083A09124070E941D13E09324071FC0C1
:10096800E43071F4E0918B07F0E0E357F84FA88189
:10097800A083A0918B070E941D13E0938B070FC0E3
:10098800E53069F4E091F207F0E0EC50F84FA88107
:10099800A083A091F2070E941D13E093F20721960D
:1009A8000895E0915C0BEA930E94F30BE0915D0BD4
:1009B800EA930E94F30B0895F4DF0E943A130E9411
:1009C8003A13E881F9810E9444130C9458091A9348
:1009D8000E94C70B1E2F103021F0E12FE150E09349
:1009E8005B0BDFDFE0915B0BEF5FF0E00E944413ED
:1009F8001991089528970E94CE1550E00E948A0BFD
:100A0800E13010F40C942606E0915C0BE43411F00C
:100A18000C947F05E0915D0BE33221F40E94C70B33
:100A2800E0935306E0915D0BE33549F4E5E5F2E028
:100A38000E944C1349DFE05DEA930E94F30BE091BA
:100A48005D0BE03511F00C947E05E2E2EA930E941A
:100A58007E0BE03019F0AF85A13009F04BC020E0E3
:100A68000E945013A03240F00E945013A23221F08D
:100A78000E945013AB3309F43DC0E22FE03071F40B
:100A88000E945013A33211F421E007C0E0915306ED
:100A9800E09355060E9456132BDF29C0E13049F434
:100AA8000E945013A43211F422E001C020E010E0AB
:100AB8001EC0E23011F0E330D1F40E9456139EDEDE
:100AC800EF3FA1F0E12FE295E07F4E2F0E945613F1
:100AD80095DEE40F1E2F2F5F243039F4E091530682
:100AE800E09355061A9304DF20E001C020E00E943D
:100AF8005D13B6CFA4C0E63511F00C940A06E09158
:100B08005D0BE334C9F50E94C70BE058FF4F1E2F59
:100B180030E0303188F50E946013E156F44FE081EF
:100B28001E1741F5AFEDBBE0EE27A30FBE1FAC913A
:100B3800A230D9F4E8E5F2E00E944C13E12F0E94BC
:100B480063130E946913AFE4BCE00E9460130E9423
:100B58006D130E9474130E946913AFE6BCE00E94F3
:100B680060130E946D130E9444130E9460130E9438
:100B7800781302C03F5FCDCFE0915D0BE33511F0F4
:100B88000C9409060E94C70BE093970B0E947D13F3
:100B9800E1F50E94C70BE093980B0E947D13A9F51D
:100BA8000E94C70BE093990BE03019F0E1E0E09365
:100BB800990B0E947D1349F50E94C70BE0939B0B8C
:100BC800F0939C0B0E947D1301F50E94C70BE093E4
:100BD8009D0BF0939E0B0E947D13B9F40E94C70BE6
:100BE800E058FF4F1E2FEE85E0939A0BE0E0EA9362
:100BF8001A930E949E0FE03041F4E8E5F2E00E946B
:100C08004C130E9483130E94441319C0E934B9F4A9
:100C1800E0915D0BEC3499F4EBE5F2E00E944C13A3
:100C2800E091920B0E948613E091930B0E94861329
:100C3800E091940BF0E0FA93EA930E94310C0E9441
:100C48006B0BDCCE0E948C13609608950E94CE1523
:100C58000E948A0BE13010F40C940107E0915C0BC0
:100C6800E33211F5E0915D0BEC3431F4E4E0E0930C
:100C7800E10CE0E0E093760BE0915D0BE43599F44C
:100C8800E091760BE03029F0EF77A0E0B0E00E9429
:100C9800B9150E94ED120E941615E0E0E093760B5C
:100CA800E7E0E093E10C04C0E43511F00C94FE0693
:100CB800E0915D0BE33231F40E94C70B3197E0936A
:100CC8005B0B98C0E03511F00C94FE0610E00E9412
:100CD8005013A03250F00E945013AD3331F00E94EF
:100CE8005013AB3311F01E3008F00CC00E94831370
:100CF800E25AF44F0E949513D001EC931F5F0E94B3
:100D08005D13E5CF0E948313E25AF44FA0E0A0835D
:100D1800EDE3EA930E947E0BE13011F00C94FE069D
:100D2800E4E5E093720B10E00E9483130E949C1389
:100D38003496E491EF3F11F40C94FE060E94A1133F
:100D48000E9483130E949C130E949115FA93EA93C0
:100D58000E942611E03011F00C94FC060E948313C7
:100D68000E949C133496E491E03839F40E94C70B32
:100D7800E058FF4FE093760B3BC0E03011F0E130D4
:100D8800A1F40E9483130E949C1332960E9491152D
:100D9800FF93EF930E94C70BAF91BF910E94B915C3
:100DA8000E94ED120E94161523C0E23081F40E94C1
:100DB80083130E949C1332960E949115FF93EF9320
:100DC8000E94C70BAF91BF910E94B11511C0E330CB
:100DD80079F40E9483130E949C1332960E94911505
:100DE800FF93EF930E94A60BAF91BF910E94B91594
:100DF8001F5F9ACF0E946B0B2BCF0E948C132696F5
:100E080008950E94D0150E948A0BE13010F40C94CA
:100E18007A07E0915C0BE332A9F4E0915D0BE035D1
:100E280019F4EEE5F2E009C0E83419F4EFE7F2E06E
:100E380004C0E33531F4EAE9F2E0FA93EA930E9458
:100E4800040C51C0E43511F00C947707E0915D0B68
:100E5800E43231F4E5E1F0E0FA93EA93ADDD43C022
:100E6800E33211F4B4DD3FC0E035E9F59ADDA09135
:100E78005B0BA531C0F50E94A6130E9491150E9434
:100E88004C13EDE3EA930E94F30B0E94A6133496E9
:100E9800E491E03829F40E9422130E94AA1323C087
:100EA800E03011F0E13049F40E94A6130E94AC131F
:100EB8000E94A5150E94AA1316C0E23049F40E94A8
:100EC800A6130E94AC130E94A1150E9474130BC0B4
:100ED800E33049F40E94A6130E94AC130E94A515A2
:100EE800EA930E943F0C0E946B0B8DCF0E94B113B6
:100EF800E0E0EC930E94D715249608951A930A937C
:100F080000E0A0915808A13081F40E94F212EE5F2F
:100F1800FA4FE081E33049F40E94F212EB5FFA4F96
:100F2800E381A0915E0AEA1709F03FC00E94B61358
:100F380001E00E948A0BE130A0F1E0915C0BE23401
:100F480079F5E0915D0BE13459F50E94C70B1E2F2E
:100F58000E94F212ED5FFA4FE081E09355060E947D
:100F6800F212EC5FFA4FE081E73419F41A930E9409
:100F780087020E94F212EC5FFA4FE081E33419F421
:100F88001A930E94C1020E94F212EC5FFA4FE081AC
:100F9800E53419F41A930E94E202EEE1E0930105A8
:100FA800C8CF0E94F2120E94FF12E02F0C94C40BCB
:100FB8001A930A930E94B61371DCE23078F10E940A
:100FC800BD130E94C3130E94D0130E94B113E2E71D
:100FD8000E94D713E0915E0A0E94DB130E94DD1382
:100FE800A0915E0AE0910A0DEA1721F4E0915E0AE9
:100FF800E03311F401E001C000E0E0915E0AE09303
:101008000A0D0A93E0915C0AEA93F4DC0E94E0136B
:101018000E94BD130E94E4130C94C40BE0E00C94EE
:10102800C40B1A93EBE5F9E00E94F113EBE5F8E045
:101038000E94F6130E94E0130E94FB13E181E4343E
:1010480071F40E94FB1302800E942213E05DE015F8
:1010580029F00E94FB13E281EA3209F401C028C09A
:101068000E9400140E94FB13E1810E94DB130E947E
:10107800FB13E2810E94DB130E9403141C910E945F
:10108800FB1333960E94F613E12FE23139F40E94E4
:10109800B1131397E6E0EC93D9DD08C0E13131F4E0
:1010A8000E94B1131397E2E1EC93ABDE0E945B0C54
:1010B8000C94230C1A93F2DBE23058F10E94BD1312
:1010C8000E94C3130E94D0130E94B113EAE70E9442
:1010D800D713EFE5FAE00E94F6130E940314119764
:1010E8001C91E12FE23131F4E6E0EA930E94F30B20
:1010F800ADDD07C0E13129F4E2E1EA930E94F30B88
:1011080080DE0E94E0130E94BD130E94E4130C9439
:10111800230CE0E00C94230CEFEFE093720BE093C8
:10112800730B0895AC81A03310F0AA3308F006C001
:101138000E940814E0530E9410140FC0AC81A1341F
:1011480010F0A73408F006C00E940814E7530E9464
:10115800101403C0A881B981E0E0EC9325960895A6
:10116800EDC2AA93EA93FA93EFB7EA931A930A9314
:101178001BB10CB1E0914A0DF0E0E85EF24F00833C
:10118800A0914A0DAF5FA0934A0DA23319F4E0E095
:10119800E0934A0D099119915CC21A93E0914B0DA5
:1011A800A0914A0DEA17D1F3F0E0E85EF24F108102
:1011B800A0914B0DAF5FA0934B0DA23319F4E0E063
:1011C800E0934B0DE12F3BC3E0914B0DA0914A0DED
:1011D800EA1709F0B3C2B4C2A091B10DBB27E091E0
:1011E800B00DF0E031960E943513EC59FF4FDF0146
:1011F800E4E6F0E00E94711508950E94D712E0918C
:10120800B10DA091B00DEA1741F0A0915706A0309A
:1012180019F0A6DFE03009F001C011C0E091B10D6E
:10122800F0E0E45BF24FE081ECB9A091B10DAF5F63
:10123800A093B10DA43619F4E0E0E093B10DE99163
:10124800EFBFF991E991B991A99199918991799112
:101258006991F9901990099018951A93E091B10D38
:10126800A091B00DEA1751F45D9B08C0A0915706F4
:10127800A13019F475DFE03009F013C01091B00DFA
:101288000E948313E45BF24FA981A0831F5F143689
:1012980009F410E0E091B10DE117E1F31093B00DFE
:1012A80002C0E981ECB91881229608950E94D015F0
:1012B8008BDFE03021F0A0915A08A03009F0C6C0B9
:1012C8006CDF1E2FA091160DA53618F0E0E0E09314
:1012D800120D3091120DE091120DE03059F41130D9
:1012E80019F4E4E0E093120D1A3519F4EBE0E093F9
:1012F800120DA4C0E43089F4E0E0E093120D1093DD
:101308005B081093140DE6E0E093120DE0E0E09323
:101318005A08E1E0E093130D91C0E53091F4E0E064
:10132800E093120D0E942213E05DE11749F00E943C
:1013380019140E9420140E942714E6E0E093120D6D
:101348007DC0E63091F40E9420140E9419141330D5
:1013580049F4E7E0E093120DE0E0E093150D0E94F8
:101368002D1402C00E94271469C0E73011F0E8303C
:1013780059F41A93E5E1FDE0FA93EA93E2E1FDE01E
:10138800FA93EA93CFDE5AC0E93081F4E0E0E093C3
:10139800120D173131F4E091150DA091140DEA17D3
:1013A80009F003C0E4E5E0935A0848C0EB3069F45B
:1013B800103039F4ECE0E093120DE0E0E0935A08C5
:1013C80003C0E0E0E093120D39C0EC3049F410930B
:1013D800170D1093140DE0E0E093130DEDE02CC011
:1013E800ED3011F50E9420140E9427140E94191450
:1013F800E091170DE150E093170DE030A1F4E09172
:10140800140DE03069F4EEE0E093120DE091130D55
:10141800E1500E943514A0E0A0830E942D1403C05F
:10142800E0E0E093120D0AC0EE3041F41D3019F4EB
:10143800EAE5E0935A08E0E0E093120DE091120D1E
:10144800E31719F0E0E0E093160D32CFDEC2AA935D
:10145800BA93EA93FA93EFB7EA931A930A9310911F
:101468009B0000919C00E12FEC71A9F4E0917A0EA9
:10147800F0917B0EEE54F24F0083AAE7BEE00E9483
:101488002F13E83CA0E0FA0731F4E0E0F0E0E09345
:101498007A0EF0937B0E09911991E991EFBFF991BA
:1014A800E991B991A99118951A930E9439140E944B
:1014B8003E14D9F30E943914EE54F24F1081ACE770
:1014C800BEE00E942F13E83CA0E0FA0731F4E0E008
:1014D800F0E0E0937C0EF0937D0EE12FB0C10E9406
:1014E80039140E943E1409F029C12AC10E94D0155E
:1014F800F6DFE03021F0A0910F0DA03009F08AC08E
:10150800D3DF1E2FA091100DA53618F0E0E0E09370
:101518000B0D30910B0DE0910B0DE03031F41130D3
:1015280019F4E4E0E0930B0D6DC0E430C1F4E0E0A1
:10153800E0930B0D1A3229F00E942213E05DE117A7
:1015480069F410935B0A10930D0DE5E0E0930B0D21
:10155800E0E0E0930F0DE1E0E0930C0D53C0E530BF
:10156800A9F4E0E0E0930B0D0E942213E05DE1177F
:1015780061F00E9445140E944C14E0910C0DEF5F3D
:10158800E0930C0DE6E0E0930B0D3CC0E630D1F49F
:101598000E944C140E944514133071F4E7E0E09364
:1015A8000B0DE0E0E0930E0DE0910C0DF0E0E55A34
:1015B800F54FA0E0A08305C0E0910C0DEF5FE0932C
:1015C8000C0D20C0E73011F0E83059F41A93EEE022
:1015D800FDE0FA93EA93EBE0FDE0FA93EA93A2DDEB
:1015E80011C0E93079F4E0E0E0930B0D173131F4E4
:1015F800E0910E0DA0910D0DEA1709F003C0E4E586
:10160800E0930F0DE0910B0DE31719F0E0E0E09384
:10161800100D6ECFFAC1AA93EA93FA93EFB7EA9343
:10162800E091810FA091800FEA1781F0E0915908AD
:10163800E03019F0E89421F808C00E9453140E9481
:10164800611419F4E0E0E093810F03C0E89420F8F6
:1016580021F8E991EFBFF991E991A9911895E881ED
:10166800A091110DEA0FE093110DE091800FF0E0C9
:10167800E058F14FA881A083E091800FEF5FE093DD
:10168800800F0E94611419F4E0E0E093800FB6C067
:10169800E0E0E093810FA091800FA13020F00E943C
:1016A8005314689421F80895AA93BA93EA93EFB76C
:1016B800EA93E0E0E093810F0E942213EF5FE0934A
:1016C8005908E991EFBFE991B991A99118950E943C
:1016D8005013A03220F00E945013AB3309F403C01A
:1016E8000E945D13F4CF0E945013AB3311F40E9493
:1016F8005D1308950E945013E881EA1729F40E94A7
:101708005D133197E1E07AC0E0E078C00E945013A1
:10171800A03228F00E94FB13E181E03208F410C0E7
:101728000E940314EC91E0935C0B0E945D130E94ED
:101738000314EC91E0935D0B0E945D13E1E00895C2
:10174800E0E008951A930A9310E00E9403140C91A4
:101758000B3311F0003208F412C0013310F00933D2
:1017680008F007C0E02FE053F0E0E457FF4FE491A2
:101778001E2B0E945D130E9403140C91E9CFE12FE8
:101788000991199108950E94D01500E010E00E9477
:101798005013AD3229F40E945D132FEF3FEF02C0C2
:1017A80021E030E00E945013A03320F00E94501333
:1017B800AA3308F00FC0D801EAE0F0E00E94431510
:1017C8000E949513E053F0E0E00DF11D8F010E9497
:1017D8005D13E8CFF901D8010E94431516C1E881CD
:1017E8000E94DB13E881A091770BEA0FE093770B57
:1017F800E881A091780BEA27E093780B2196089569
:101808001A9310E00E946614E03031F00E946614CA
:10181800EA93E5DF1F5FF6CF2BC01A9310E00E9412
:101828008313E25AF44FE081E03049F00E948313B9
:10183800E25AF44FE081EA93D2DF1F5FF0CF1991AB
:1018480008950E94A113E6EBF2E0FA93EA93EC8183
:10185800FD810E946E140C947F101A930E94A113AC
:10186800E9EBF2E0FA93EA93ED81FE810E946E14AF
:101878001881239608951A93ECE3EA93B0DF11E0F8
:10188800193080F40E948313E457FF4FE491A98133
:10189800EA2319F0E12FE05D01C0E0E2EA939FDF5F
:1018A8001F5FEECFEEE3EA939ADF0C947E101A9353
:1018B8000A93E0915B09E03011F40C94BD10EAE55D
:1018C800EA93CBDCE0E0EA93C8DC10E00E948313E3
:1018D800E55AF64FE081E03011F01F5FF7CF1F5F48
:1018E800012F0A93BADC10E00E948313E55AF64FE1
:1018F800E081E03079F00E948313E55AF64FE081E9
:10190800EA93ABDC0E948313E55AF64FE0810E0F91
:101918001F5FEACFE02FE195EA939FDCEDE0EA93C1
:101928009CDC0C94BD100E94D015AC81BD81EC915B
:10193800E03021F40E94D7150C942411E0E0E093E4
:10194800800FE1E0EA938BDEE0E0E093110DAC81DB
:10195800BD81EC91E03041F0EA9381DEEC81FD81BC
:101968003196EC83FD83F3CFE3E0EA9378DEE091F0
:10197800110DE295EF70EA930E9416040E2FE09184
:10198800110DEF70EA930E9416043E2F0A9367DE4A
:101998003A9365DEE7E1EA9362DE689420F80E94F4
:1019A800D7150C9424110E94D01580DCA0915A08F8
:1019B800AA3511F40E941508A0915A08A43511F50A
:1019C80000E00E94BD13EB5FFA4F9F01E02F0E94D9
:1019D8003514E081E03051F0E02F0E943514E081A9
:1019E800D901EC930F5F2F5F3F4FF0CFD901E0E0B3
:1019F800EC930E94BD130E947814E0E0E0935A082B
:101A0800E12F03C0E0E0E0935A080E94D71524961E
:101A180008950E94CE156ADDA0910F0DA43511F02E
:101A28000C94900D10E0A0915B0AAA3221F4E09189
:101A38005D0AED3409F050C0E7E0E093E10CE09175
:101A48005E0AEA35D9F500E04FEF5FEFE091600AF2
:101A5800E7703E2FE0915F0AE23361F4A4E1B0E061
:101A68000E94A515AE2F0E946013E457FF4FE49122
:101A7800EA2309F414C0E1E6FAE00E94F6130E9492
:101A88005013AB3421F40E945D137DDE0E2F0E94AB
:101A98005013A43521F40E945D1375DEAF01009345
:101AA8000005E8ECF0E0E093950BF093960B40937B
:101AB800E50C5093E60CE2E0E093E10CE0915E0A5D
:101AC800E03519F4E1E0E093E10CE0915E0AE234DC
:101AD80019F4E1E0E093E10C0E942213E05DA0918B
:101AE8005B0AEA1799F4E0915D0AE23521F40E9455
:101AF800DC071E2F0BC0E23721F40E9482071E2F3D
:101B080005C0EA3519F40E945E081E2FE0E0E09354
:101B18000F0DE12F0C942211E0E00C942211A0E0AB
:101B280020FCA1E0A13049F4A0E021FCA1E0A03014
:101B380021F4A0915908A03009F001C0A9DDE09175
:101B48005908E03019F0E150E09359080895A88148
:101B5800A13118F0E881E051E883E8810E948414FB
:101B6800A091DC0FB091DD0FEA2BFB2BE093DC0F8B
:101B7800F093DD0F0C9451111A930A9310E0103171
:101B8800D0F40E9483130E947813AFEBBBE0EE27DA
:101B9800A10FBE1FEC93AFECBBE0EE27A10FBE1F59
:101BA800EC93AFE0BCE00E9483130E948E140E9465
:101BB80093141F5FE4CFDDC20E94D015E0917D0B26
:101BC800F0917E0BAC81BD81EA27FB279F0110E0D5
:101BD800123190F4F901E17039F0A12FB0E0A0586A
:101BE800B44FEC91EF5FEC93D901E2E0F0E00E9492
:101BF80069159F011F5FECCFEC81FD81E0937D0BA0
:101C0800F0937E0B0E94D7151BC30E945204E0304C
:101C180061F10E94BD13EB5FFA4F0E94F113AFEA26
:101C2800BBE0E881F0E0AE0FBF1FEC910E94DB1330
:101C38000E942213E05D0E94DB130E94B113E2E5CB
:101C48000E94D7130E9498140E94DD13E4ECF2E07E
:101C58000E944C13E8810E94A4140E9463130E94FE
:101C6800E0130E94BD130E9478140C9451110E9435
:101C78005204E03069F10E94BD13EB5FFA4F0E94F5
:101C8800F113A5E1B0E00E94A515E05D0E94DB1309
:101C98000E942213E05D0E94DB130E94B113E2E56B
:101CA8000E94D7130E9498140E94DD13E7ECF2E01B
:101CB8000E944C13E9810E94AA130E946913E881CB
:101CC8000E94AA130E94E0130E94BD130E94781478
:101CD80012C20E94CE15A091950BB091960B0E944E
:101CE800CA1524F4A5E9BBE00E94A914E091950B5C
:101CF800F091960B309719F4E0E0E093000510E0BE
:101D0800123110F00C94D20EA12FB0E0AF5FBF4F8C
:101D18000E94A515E13011F00C94D00E0E94831397
:101D2800E653F04F0081E12FE695E695E6952E2FD4
:101D3800E12FE770EF5F5E2FE22FF0E0EE56F44FF1
:101D48001080E52F0E948414A12DB0E0EA23FB2324
:101D58003097B9F40A3821F40E945204E03009F4AB
:101D680006C0E12FEF5FEA93E0E0EA9380DF0038F6
:101D780010F00B3808F001C00F5F003209F400E8DA
:101D880006C0003208F40F5F013808F000E00E9436
:101D98008313E653F04F00831F5FB2CFE0E0F0E01B
:101DA800E093DC0FF093DD0FE093E40C00E00031EA
:101DB80010F00C94950FE02F0E94A414E03011F459
:101DC8000C94930FE091E40CEF5FE093E40CAFED1B
:101DD800BBE00E94AF14E03079F40E94B4140E9472
:101DE8008E140E94A9140E94B4140E946D13309797
:101DF80011F40E94B91475C0E13011F00C94520F1F
:101E08000E94BF14E1501E2F0E948313E058F44F24
:101E1800E081E030A9F40E94C2140E942F130E94AE
:101E2800C714309749F00E94C2140D901C900E946C
:101E3800C714E015F1050CF002C00E94B91419C0CE
:101E48000E94B4140E94CC14BF010E94B4140E94D2
:101E58006D13DF010E9483130E94D1140E94351371
:101E6800DB010E94D6140E94D9140E94C2140E9459
:101E780093140E94B4140E946D13FF2332F40E943D
:101E8800B4140E948E140E9493140E94B4140E94E9
:101E98006D13309711F40E94B91423C0E23009F58C
:101EA8000E94BF14E1501E2F0E94DE140E94CC1421
:101EB8000F010E94DE140E946D13DF010E9483133C
:101EC8000E94D114EA0FFB1FD0010E94D6140E9471
:101ED800D914AFE4BCE00E94E3140E948E140E945F
:101EE8002F130E94BF14EA9332DEAFEFBBE00E94CB
:101EF800AF14EA932CDE0E94E6140E946D1330970B
:101F080071F00E94E6140E948E140E94A9140E9487
:101F1800E6140E946D13309711F40E94B9140F5FF4
:101F280046CFE091DC0FF091DD0FE093DF0CF093EA
:101F3800E00C84C10E94D01530E010E0103168F444
:101F48000E948313E156F44FE081AE2FEC81EA172B
:101F580011F431E002C01F5FF1CF303071F410E0AE
:101F6800103158F40E948313E156F44FE081E030B9
:101F780011F431E002C01F5FF3CF313011F00C943F
:101F88004F10AFEEBBE00E948313EA0FFB1FA09136
:101F9800970BA083AFEFBBE00E948313EA0FFB1FF0
:101FA800A091980BA083A091E20CA23051F4AFED60
:101FB800BBE00E948313EA0FFB1FA091990BA0833B
:101FC80007C0AFEDBBE0EE27A10FBE1FE2E0EC9328
:101FD800AFEEBBE0EE27A10FBE1F2C91213070F0B1
:101FE800E22FE150F0E00E94D914E22FE150A6EA76
:101FF800BFE0F0E00E948E140E949314AFE0BCE0B2
:102008000E9483130E94CC14A0919B0BB0919C0B4F
:10201800A083B183AFE2BCE00E9483130E94CC147A
:10202800BF01A0919D0BB0919E0BE4E6F0E00E94E9
:102038004315DB010E94D614E156F44FAC81A0830E
:10204800AFEBBBE00E948313EA0FFB1FA091E70CE4
:10205800A083AFECBBE00E948313EA0FFB1FAD81A6
:10206800A083AFE4BCE00E9483130E948E140E94F8
:102078009314AFE6BCE00E9483130E948E140E9462
:102088009314AFEABBE00E948313EA0FFB1FA091F1
:102098009A0BA08331E0E32F0E94D715D1C01A9381
:1020A80010E0103490F4E12FAFE9BBE0F0E00E94BB
:1020B8008E140E949314AFE1BCE00E9483130E9427
:1020C8008E140E9493141F5FECCF10E0123130F48D
:1020D8000E9483130E94D9141F5FF8CFE981E03072
:1020E80009F406C0A091E30CAF5FE3E00E946E150F
:1020F800E093E30C1881229608953EDD0C9451116B
:102108001A930A93E091E20CA091E10CEA1789F086
:102118000091E10C073009F42FDD013019F4E0E0FB
:10212800EA93BDDF023019F4E1E0EA93E6DF0093B9
:10213800E20CA091E20CA73019F4E0E0E0937F0BE9
:10214800A091E20CA13019F4E0E0E0937F0BA0919C
:10215800E20CA23071F4A0910005A13020F0A0910A
:10216800E60CAA230AF402C0E1E001C0E0E0E09333
:102178007F0B0991199108950E94CE15E7E0E0932D
:10218800E10C10E0153110F00C9422110E94831319
:102198000E949C1332960E9491159F010E948313FE
:1021A8000E949C1332960E949115AF010E948313DE
:1021B8000E949C133496E491E03011F0E130B1F4C0
:1021C800D9010E94A515AE2F0E9483130E949C136B
:1021D8003596E491EA1748F40E9483130E949C13F1
:1021E8003696E491D9010E94B91526C0E230A1F4CF
:1021F800DA010E94A115E031A7E2FA0714F4FF23DF
:1022080052F40E9483130E949C1336960E949115E3
:10221800DA010E94B11510C0E33071F4D9010E94AF
:10222800A515EF3F49F40E9483130E949C1336962C
:10223800E491D9010E94B9151F5FA4CF0E94D5155A
:1022480026960895E991F991A991B9911D90059063
:10225800011421F40020D1F7EE2708951018E1F3B6
:10226800E1E008F4E2500895A991B991EE27FF271B
:102278006D91662311F03196FBCF0895AA27BB27ED
:10228800E991F9910590002011F01196FBCFFD011D
:1022980008955D9BFECFE881ECB9219608951A93C5
:1022A8000A93AC81BD810E948D153097C1F0AA8137
:1022B800BB810E948D158F01309749F00230E0E014
:1022C8001E0760F0F80131978F01ED93FC93AC8104
:1022D800BD810E942F133197AE81A08303C0EE8188
:1022E800EA93D7DF198108812796089526970E94D7
:1022F800CE1510E0EA89FB893196EA8BFB8B319782
:10230800E4912E2FE03011F40C94A612E12FE03066
:1023180039F4253211F411E002C00E94E91411C108
:10232800E130A9F4253219F40E94E91409C112E038
:1023380040E000E02D3211F401E003C12B3211F42A
:102348004BE2FFC0203211F440E2FBC002C0E23091
:1023580039F450E013E0203311F40068F2C004C0EF
:10236800E33011F00C94A512203310F02A3308F052
:1023780009C0A52FEAE0EA9FF0015E2FE22FE053A3
:102388005E0FDFC0E22FE33649F40E94F414E889B7
:10239800F989A481AA930E94FA14D2C0E33741F4C0
:1023A8000E94F4140E9404150E9438111E2F0AC0BE
:1023B800E03761F40E94F4140E9404150E9442114F
:1023C8001E2F086002600F7730E035C0E43611F048
:1023D800E93611F4046002C0E53731F4E6E3F2E0CF
:1023E800EE83FF8315E00DC0E83511F4086004C0E2
:1023F800E83711F00C94A412E0E4F2E0EE83FF83D6
:1024080014E002FF14C00E94F4140E940E15AB855C
:10241800AA233AF4EA85FB850E942615EA87FB87FA
:102428004DE2403011F01F5F01C00B7F04C00E94D5
:10243800F4140E940E1500FD11C0151778F407FF5B
:1024480008C002FF04C00B7F242F115001C020E3F5
:1024580001C020E20E94E9145150EFCF312F01FF53
:102468001AC03030B9F003FF08C0EE81FF81319601
:10247800EE83FF833197E49105C0AE81BF81ED9172
:10248800AE83BF83EA930E94FA14503009F051508A
:102498003150E7CF4BC020E3EE81FF810E949115B8
:1024A800E887F987EE81FF813296EE83FF83E8851E
:1024B800F985AA85BB85AE17BF0750F02F5FA885A1
:1024C800B985EA85FB85EA1BFB0BEA87FB87EFCF1B
:1024D8002A3328F003FF02C0295F01C0295D04FDEB
:1024E8001AC0213320F4A885B985119709F409C0C9
:1024F800531710F000FF01C013C020E207FF0BC004
:1025080020E3006102FF07C00B7F4A930E94FA1480
:10251800503009F051500E94E914503009F05150E0
:102528003150A885B985129708F0B5CF00FF08C0CB
:10253800503031F05150E0E2EA930E94FA14F8CF9B
:1025480010E0D8CE0E94D51564960895FF92F82E13
:1025580022971A930A93DE010E9422158D01DE014B
:1025680016960E9422150E948D15EA83FB83DE01D0
:1025780014960E9422150E948D15FA93EA931A93D5
:102588000A93FE013696FA93EA93E0E0F0E0FA93B4
:10259800EA93ACDEAA81BB81E0E0EC931981088163
:1025A8002496FF9008950A921A92FA926A937A935F
:1025B8008A939A93AA93BA93EA93FA93EFB7EA9312
:1025C8000895E0915206EA930E944804E093520667
:1025D8000895EAE0F0E0FA93EA930895E09152064C
:1025E800A3E4EA9FF0010895EB5FFA4FFA93EA93A8
:1025F8000E94970CF3CFEE5FFA4FA0E0A083E1CFE3
:10260800EA930E941604EA930C947C04E8EEFCE03A
:10261800E093060DF093070D0895A091060DB09173
:10262800070D0895A091060DB091070D1796EC932C
:102638000895AF5FE4E60E946E150895A0E0B0E04B
:102648000E94A5150895E0936500E6E9F0E0FA9385
:10265800EA930C941615ED91FD913196FE93EE9345
:1026680008950E949A15EA1BFB0B0895E881F981E9
:10267800FA93EA930E94250CECE2EA930C94F30B8C
:10268800FA93EA930E94250CEBE3EA930C94F30B7C
:10269800FA93EA930C94040CA0917B0BB0917C0BF9
:1026A800AC910895A0917B0BB0917C0BEC91EA93CF
:1026B8000895ABE7BBE0CFCFE32FF0E00895EF77C5
:1026C800F0E0FA93EA930C94250CEAE3EA930C946D
:1026D800F30BEE0FFF1FAE0FBF1F0E948D1508955D
:1026E800FA93EA930C94250CE156F44FA0E0A083EA
:1026F8000895EAE3EA930E947E0BE1300895E12F02
:10270800F0E00895F0E0FA93EA930E94310CDDCFEF
:10271800A091790BB0917A0BE0E0EC930E94D5156B
:1027280008950F01A0917B0BB0917C0BEC9108955B
:102738000E942A15EA56FF4F0895EEE5FBE0FA934A
:10274800EA930895E0915B0BF0E0F2CFF0E0C8CF98
:1027580032960E949115DF010895A091790BB091EE
:102768007A0B0895E0E6FAE0E0937B0BF0937C0B9C
:102778000895E0915106A3E4EA9FF0010895EB5F04
:10278800FA4FE093790BF0937A0BE0915C0AE5DF5E
:10279800EC93A9E7BBE05FCFE0915B0ADEDFEC9347
:1027A800A9E7BBE058CFEC93A9E7BBE054CFD5DF4E
:1027B800FACFD3DFEFE0F7CFD0DFE0E0EC93089576
:1027C800EE5FFA4FA1E0A083E0915106EA930E94E0
:1027D8004804E0935106E1E00895E093790BF09303
:1027E8007A0B0895E0937B0BF0937C0B0895E091AE
:1027F8007B0BF0917C0B0895A9E7BBE02CCFA0914F
:102808007B0BB0917C0B0895AA81BB81EC91E2957A
:10281800E07FAE2FEC810895EA0FAA81BB81EC938B
:10282800A881B981EC91EF5F0895E12FA091140D73
:10283800EA0FE093140D0895E091130DF0E0E55AC6
:10284800F74F10830895E091130DEF5FE093130D98
:102858000895E091130DF0E0E55AF74FA0E0A0834A
:102868000895F0E0E55AF74F0895E0917C0EF09155
:102878007D0E0895A0917A0EB0917B0EEA17FB07A2
:102888000895E12FA0910D0DEA0FE0930D0D089525
:10289800E0910C0DF0E0E55AF54F10830895E091B2
:1028A800810FF0E0E058F14FE081E0939C00E09167
:1028B800810FEF5FE093810F0895F0E0E030A1E031
:1028C800FA070895E12FA981BA81F0E0EA0FFB1F0A
:1028D800E49108950E9436150E94951584E00E949F
:1028E800AA1228960C94110CEE5FFA4FA1E0A0836F
:1028F800E0915106EA930E944804E0935106089536
:10290800A6E4B1E0F0E0EE0FFF1FEA0FFB1F0E9404
:1029180091150895EE0FFF1FAE0FBF1F0895E0E059
:10292800F0E0ED93FC930895E0915606E05D15DF25
:10293800EC93E0915606EF5FE770E09356065CCFA4
:10294800F0E0E156F44FE0810895ED91FD91319763
:10295800FE93EE930895EE27A00FBE1FEC91089505
:10296800AFE0BCE0E02FF0E008950A930E94090E62
:10297800E02FF0E0B9CEAFEEBBE0EDCFE12FA6EA55
:10298800BFE0F0E0C7CFE12FA2E8BFE0F0E0A1CEC2
:10299800EE0FFF1FEA0FFB1F0895E058F44FE08188
:1029A800F0E00895ED93FC93AACEE058F44FA0E030
:1029B800A0830895AFE6BCE0E02FF0E00895E02F93
:1029C800F0E00895AFE2BCE0FACF2A93EF85F889EA
:1029D800FA93EA93FE013F96FA93EA930C94531103
:1029E800E889F9893497E88BF98B0895EF85F88998
:1029F800FA93EA93FE013F96FA93EA930C945311E3
:102A0800A889B98914960E948D15EE83FF83FA93DD
:102A1800EA930895A889B98914960E948D15EA87C2
:102A2800FB870895E991F991309639F080EA9FE0A3
:102A38000197F1F7A8953197C9F708950024AF0DCC
:102A4800B01D0895F195E195F0400895EE0FFF1F30
:102A5800EE0FFF1FEE0FFF1F0895EF2FFF27E7FD73
:102A6800FFEF08956F2F660F660B762F0895FA9F74
:102A7800F02DEB9FF00DEA9FE02DF10D08953BD06E
:102A8800F6DF0EF4DFDF0895002498E0AA0F001C9B
:102A98000E1A10F40E0E01C0A1609A95B9F7EA2F2C
:102AA800A02D08950024112490E1AA0FBB1F001C3B
:102AB800111C0E1A1F0A18F40E0E1F1E01C0A16069
:102AC8009A9599F7FD01D001089515D0EBDF0EF422
:102AD800B9DF0895D9DFEA2F0895E894B7FF04C055
:102AE800A095B09511966894F7FDACDFDBDFFD018A
:102AF8000EF4A8DF0895E894F7FF02C0A3DF6894F6
:102B0800B7FF06C0A095B095119600F8039400FA97
:102B18000895ED91FC91119708950590F491E02D99
:102B280008957A936A93FA93EA9308951B2EBF2F18
:102B3800F12D1A2EAE2FE12D0895119602D0FE2FF9
:102B48001197E199FECFFF93FFB7F894AEBBBFBBD7
:102B5800E09AEDB3FFBFFF91089507D01196EF9368
:102B6800EF2F03D0EF9111970895E19B02C0A8952C
:102B7800FCCF9FB7F894AEBBBFBBE09A8DB3E81704
:102B880019F0EDBBE29AE19A9FBF089500240A1656
:102B98000B0608955A934A933A932A931A930A93E1
:102BA80008955D814C813B812A81198108810895AE
:00000001FF
